:100000001CC035C034C033C032C031C030C02FC076
:100010002EC0C1C02CC02BC02AC029C028C027C0F8
:1000200026C025C024C052C055C059C05DC063C0A1
:1000300067C06DC073C077C042C011241FBECFE53A
:10004000D4E0DEBFCDBF10E0A0E6B0E0EAE9F7E023
:1000500002C005900D92A036B107D9F710E0A0E6D6
:10006000B0E001C01D92A837B107E1F76FC1C8CF5A
:10007000CF93DF9324E630E0829FA001839F500D51
:10008000929F500D112420E04115510569F0A4EC18
:10009000B9E0C0E0D0E0CD010197F1F72F5F822FEA
:1000A000992784179507B8F3DF91CF910895AA2770
:1000B000BB27FC010A9748F4ED5EFF4F099482B319
:1000C000896082BB82B3897F82BB089582B3807FBF
:1000D00082BB0895909A82B3817F82BB0895919AE2
:1000E00082B3827F82BB089582B3836082BB82B376
:1000F000837F82BB0895929A82B3847F82BB0895E6
:1001000082B3856082BB82B3857F82BB089582B350
:10011000866082BB82B3867F82BB089582B387608C
:1001200082BB93980895939A82B3887F82BB089587
:100130008330910591F08430910530F48130910540
:10014000D9F00297A1F0089585309105D1F085305E
:10015000910540F00697D1F00895AA9885B38B6376
:1001600085BB0895AB9885B3876385BB0895A9982F
:1001700085B38D6385BB0895A89885B38E6385BBD1
:100180000895AC9885B38F6285BB0895AD9885B30B
:100190008F6185BB08951F920F920FB60F921124A5
:1001A0002F933F934F935F936F937F938F939F937F
:1001B000AF93BF93EF93FF9385B38F6385BB86E9BE
:1001C0008A95F1F782B3807F82BB80917100909114
:1001D0007200AEDF809171009091720083309105C2
:1001E00039F18430910570F08530910581F18530C9
:1001F000910518F18630910579F1019687309105C6
:1002000081F513C081309105E9F082309105A9F79D
:1002100080916200909163004ADF8091710090911B
:100220007200019687309105E1F481E090E019C0F9
:100230008091640090916500EFCF8091660090916D
:100240006700EACF8091690090916A00E5CF8091C4
:100250006B0090916C00E0CF809160009091610004
:10026000DBCF90937200809371008FEF82BFFF917C
:10027000EF91BF91AF919F918F917F916F915F911E
:100280004F913F912F910F900FBE0F901F90189597
:1002900060916F00862F99270196CC973CF020E063
:1002A000422F622F80916D005ED108956F5F20E034
:1002B000422F80916D0057D1089560916F00862F75
:1002C0009927019797FD07C0615020E0422F809148
:1002D0006D0049D1089520E0422F6BE380916D00BD
:1002E00042D1089530916D00832F99270196489748
:1002F0004CF0209168004091730060916F0080E0A5
:1003000032D10895209168004091730060916F0090
:10031000832F8F5F28D1089530916D00832F992707
:10032000019797FD0AC02091680040917300609189
:100330006F00832F815017D108952091680040915C
:10034000730060916F0087E10ED10895CFE5D4E08E
:10035000DEBFCDBF74D0E0D081E089BF8FEF82BF18
:1003600085E083BF789481E090E090937200809361
:10037000710081B38F6081BB84B38F6384BB28E637
:1003800030E043E750E06FE670E08DE690E087D024
:1003900020916D00822F6AE0E0D1992790936A0046
:1003A00080936900822FD9D1892F99279093630078
:1003B0008093620020916F00822FCFD19927909374
:1003C000650080936400822FC8D1892F992790936C
:1003D00067008093660020917300822FBED1992719
:1003E00090936C0080936B00822FB7D1892F99274F
:1003F000909361008093600031D0882309F4BFCFCF
:100400008091750080936E0043D080916E00992793
:100410008230910581F0833091052CF4019709F029
:10042000AECF36DFACCF8330910539F0049709F0B9
:10043000A6CF72DFA4CF41DFA2CF54DFA0CFB99AFD
:10044000BA9A0895982F80E0B69902C0892F04C007
:10045000B79902C0892F8F5F99270895BE98BF98DA
:10046000C69AC79A10927500C19881E0EBDF882385
:1004700011F080937500C19AC29882E0E3DF88236F
:1004800019F08F5F8093750080917500992708950A
:10049000E5DF8823E9F784E190E0C2D00895AF92C8
:1004A000BF92CF92DF92EF92FF920F931F935C0166
:1004B0006B017A01890125D081E051D0F801808358
:1004C00082E04DD0F701808383E049D0F60180833C
:1004D00084E045D0F501808309D01F910F91FF90F2
:1004E000EF90DF90CF90BF90AF90089525D180918D
:1004F00076008F7B809376006091760080E064D0F8
:1005000008951AD18091760080648093760060917E
:10051000760080E059D0089510927600109277000E
:1005200060E0862F51D084E008D08F73682F84E07C
:100530004BD060E988E048D008951F93182FBFD0B2
:1005400080EACDD0812FCBD0BAD081EAC8D081E06B
:1005500090D0182FBED0812F99271F910895EDDFDD
:100560004BD099270895EF92FF920F931F93E82E97
:10057000F62E042F122F1DD0612F81E034D0602F72
:1005800082E031D06F2D83E02ED06E2D84E02BD011
:1005900005D01F910F91FF90EF900895CDD08091DD
:1005A00076008F77809376006091760080E00CD0A3
:1005B0000895C2D080917600806880937600609123
:1005C000760080E001D008950F931F93182F062F17
:1005D00076D080EA84D0812F82D0802F80D079D0CD
:1005E0001F910F9108951F93182F862F0FD0682FFA
:1005F000812FEADF1F910895982F9F7002C0965FA8
:1006000080518031E0F7892F9927089590E002C04A
:10061000905F8A508A30E0F7980F892F99270895C4
:10062000CF93DF93EC0121978FEFCF3FD80741F0B5
:1006300088EE93E008D021978FEFCF3FD807C1F71E
:10064000DF91CF91089565E070E093D0CB01AA27A8
:10065000BB2723E0880F991FAA1FBB1F2A95D1F73C
:1006600020E030E002C02F5F3F4F28173907D8F352
:1006700008950F931F93CF93082F10E08E98969AAA
:1006800068D0C7E0959A65D0110F8699116095984A
:1006900060D0C150C7FFF6CF8E9A002311F4969810
:1006A00001C0969A56D0959A54D0959852D0969863
:1006B00050D0812F9927CF911F910F910895959A2E
:1006C000969A8E9A8D9A45D0969843D0959841D017
:1006D00008958E9A959A3DD0969A3BD008951F938F
:1006E000CF93182F8E9AC7E009C0969832D0959A6A
:1006F00030D09598110FC150C7FD0BC017FFF5CF33
:10070000969A27D0959A25D09598110FC150C7FF7A
:10071000F5CF8E98969A1DD0959A1BD0CFEF03C037
:1007200018D0C15011F08699FBCF959812D08C2F1C
:100730009927CF911F91089580E0FFDE8093760086
:10074000809176008270809377008091760099275F
:10075000089585E090E077DF0895991B79E004C063
:10076000991F961708F0961B881F7A95C9F78095F0
:100770000895AA1BBB1B51E107C0AA1FBB1FA617E8
:10078000B70710F0A61BB70B881F991F5A95A9F73A
:0A07900080959095BC01CD010895FD
:00000001FF
